:100000000C948E020C94C6020C94C6020C94C60288
:100010000C94C6020C94C6020C94C6020C94C60240
:100020000C94C6020C94C6020C94AA230C947C2453
:100030000C94CB1C0C94C6020C94C6020C94C60201
:100040000C94C6020C94C6020C94C6020C94C60210
:100050000C94C6020C94541D0C94C6020C94C60257
:100060000C94C6020C94C6020C94C6020C94C602F0
:100070000C94C6020C94C6020C94C6020C94C602E0
:100080000C94C6020C94C6020C94C6020C94C602D0
:100090000C94C6020C94C6020C94C6020C94C602C0
:1000A0000C94C6020C94C6020C94C602820582050A
:1000B000AE05AE050F060607060706072D069506D0
:1000C000A606A606C8163A17D0169A169E16D41675
:1000D000A116D716E216AC163017B016E616B416EF
:1000E000EA161417B816EE161E17BE16F416FE16EC
:1000F000A516DB16A816DE16C316F9160A172A1758
:100100002C179616CC164317F818FE18EC18F21890
:1001100004190A1910190D1A101A471A5A1A621AD4
:100120006D1A701A701A701AB81AB81A751A781AE5
:100130007D1A8A1A971A9A1A9E1AAB1AE4240B256A
:1001400003260B25032657257A250326D125E025EE
:100150005600540029001F0021002300250027001D
:100160002E004600550053001E00200022002400EF
:1001700026002D0031000000570060002B001A00FF
:1001800015001C000C00130030004C0061005F00E3
:10019000140008001700180012002F002A000000A9
:1001A00057005D003900160009000B000E003300F7
:1001B00028004B005E005C00040007000A000D00F0
:1001C0000F0034003500000058005A00E1001B0009
:1001D0001900110036003800520000005B00590081
:1001E0001D0006000500100037000000E5004E006D
:1001F00058006200E000E20000002C000000E40073
:100200005100000063006200E300000000000000F5
:100210002152000050004F000100010001000100C8
:1002200001000100010001000100007C010001004B
:1002300001000100010001000100010001000000B7
:1002400001000100010001000100010001000100A6
:100250000100037C01000100010001000100010018
:100260000100010001000000010001000100010087
:1002700001000100010001000100027C01000100F9
:100280000100010001000100010001000100000067
:100290000100010001000100010001000100010056
:1002A0000100000001000100010001000100010047
:1002B0000100000001000100010001000100010037
:1002C0000000010000000100010000000100010029
:1002D000010000000000000001000000010001001A
:1002E00000AE00AF00DA0281FFD9F1DB20A4A62E18
:1002F000AF00A0C0D30000A1C8D30000AED580A835
:100300001F408D14200000000000000000002A2B78
:1003100028000000000000000000000000000000B5
:100320000029000000002C1E34202122243426271E
:10033000252E362D3738271E1F202122232425263F
:100340003333362E37381F0405060708090A0B0C0D
:100350000D0E0F101112131415161718191A1B1C55
:100360001D2F3130232D350405060708090A0B0C13
:100370000D0E0F101112131415161718191A1B1C35
:100380001D2F3130354C000000000000000000003F
:10039000000000000000000000000000000000005D
:1003A000000000000000000000007E0F00D4FFFFEE
:1003B000FFC7000000780C03450078007400360089
:1003C0003500000012034100450042006F0061004B
:1003D00072006400730000000403090409025B005A
:1003E000030100A0FA090400000103010100092132
:1003F00011010001224400070581030800010904DE
:100400000100020300000009211101000122220065
:1004100007058203200001070503032000010904EA
:1004200002000103000000092111010001226D00FA
:1004300007058403200001120100020000000845A6
:100440004165AE0100010200010660FF0961A101E2
:100450000962150026FF00952075088102096315C1
:100460000026FF00952075089102C005010980A1B2
:1004700001850319012AB700150126B700950175FA
:10048000108100C0050C0901A101850419012AA0F1
:1004900002150126A002950175108100C005010911
:1004A00006A1018506050719E029E7150025019534
:1004B00008750181020507190029EF15002501952E
:1004C000F07501810205081901290595057501914D
:1004D00002950175039101C005010906A1010507F7
:1004E00019E029E71500250195087501810295019C
:1004F000750881010507190029FF150026FF0095E1
:1005000006750881000508190129051500250195C2
:100510000575019102950175039101C011241FBE5B
:10052000CFEFDAE0DEBFCDBF04B603FE18C0809186
:100530001E0590911F05A0912005B09121058730DF
:10054000904BA740B04B59F410921E0510921F0516
:100550001092200510922105E0E0F8E3099511E0E2
:10056000A0E0B1E0E6EEFDE402C005900D92AA3BEA
:10057000B107D9F725E0AAEBB1E001C01D92AE3179
:10058000B207E1F70E9459120C94F1260C94000076
:10059000519A0E94210E0895CF93C82F0E940A04F9
:1005A000813011F4599A01C059988C2F0E94B507D7
:1005B000CF9108958230B0F46A30A0F44A3090F4BC
:1005C00094E6899FF00111248AE0689FE00DF11DF7
:1005D0001124E40FF11DEE0FFF1FE05BFE4F85912C
:1005E0009491089581E090E0089581E0089581E07C
:1005F00008950E94F70208950E94F90208950E944A
:10060000F702089508950E9402030895A6E0B0E05D
:10061000ECE0F3E00C94612649835A839E83309189
:10062000C10189819A81311115C03E81332359F06E
:10063000222349F00E949908182F682F89819A81F6
:100640000E94750803C00E948708182F69817A816B
:10065000812F04C00E94990869817A810E94F90F54
:100660002696E3E00C947D26FC01262F40815181E3
:1006700062817381848195810E9406030895CF93DE
:10068000DF93EC0161E00E943403BE010E94FC0292
:10069000DF91CF910895CF93DF93EC0160E00E944A
:1006A0003403BE010E940303DF91CF91089591E0CE
:1006B00001C0990F8A95EAF7892F0E94C107089512
:1006C000CF93C82F81E00C2E01C0880F0A94EAF75F
:1006D0000E94450D8C2F0E945703CF91089581E011
:1006E00008950E946F030895CF93C82F0E94730747
:1006F0008C2F0E9471032FEF84E39CE021508040F7
:100700009040E1F700C00000CF91089581E00E9481
:1007100074030E947A1D089580E00E9474030E9471
:100720009E1D08950F931F93CF93DF938C0161E07B
:100730000E943403EC01B8010E94DA19882309F4FD
:1007400057C0B801CE010E94FF02882309F450C0AF
:10075000B801CE010E94E018882309F449C0B8010D
:10076000CE010E947216882309F442C0B801CE015E
:100770000E9448168823E1F1B801CE010E94231996
:100780008823B1F1B801CE010E94F710882381F1CE
:10079000F8018581882341F1C3308CE7D807D1F077
:1007A00040F4C115FCE7DF0791F0C130DC47A1F050
:1007B0001BC0CB35ECE7DE07A9F0CC35FCE7DF0743
:1007C00071F0CA35DC4781F40E94200D0DC00E94F3
:1007D00086030EC00E94280D0E948C0309C00E944F
:1007E000160D02C00E94240DC8010E94F50201C02E
:1007F00080E0DF91CF911F910F9108950E94A31C7B
:100800000E9449040E94461408950E944D040E94CB
:10081000AC1C0895982F92959F7019F0892F24E0B1
:1008200001C020E0982F9695969511F02E5F892FA4
:10083000982F969509F02F5F822F089581E00895F3
:1008400080FF02C05D9A01C05D9881FF02C05B9A83
:1008500001C05B9882FF02C05A9A08955A98089581
:10086000CF93DF93D82F0E941E04C82F882319F03E
:100870008D2F0E9420048C2FDF91CF910895559ADF
:100880005D98539A5B98529A5A9808950E94300442
:10089000089580E00E94460408950E94C81A0E94AC
:1008A00046040895CF930E94C81AC82F8091BC01B6
:1008B000C81779F0C093BC010E94391D6093BD0137
:1008C0007093BE018093BF019093C0018C2F0E9452
:1008D0004604CF910895ADE0B0E0E1E7F4E00C9478
:1008E0006226488759876A877B878C879D87911105
:1008F0000E94220CCE01019627E0FC0111922A955C
:10090000E9F726E0FE013896DC0101900D922A9568
:10091000E1F72D8121110AC029813A814B815C8147
:100920006D817E818F810E946C0B04C00E943F0309
:100930008111F2CF2D96E2E00C947E26FC012481F9
:10094000213021F4808191810E94C6080895CF93BF
:100950008823D9F1C82F8CEF8C0F813A70F48C2F3B
:100960000E945A1B882329F08C2F0E94FF1B0E9493
:10097000A90C8C2F0E94E51B0CC080E28C0F8830E4
:1009800058F4C77081E001C0880FCA95EAF70E9449
:10099000050C0E94A90C19C0EBE5EC0FE33040F404
:1009A000F0E0EE5AFE4F808190E00E94EE1A0DC0FA
:1009B000C85ACB3150F4EC2FF0E0EE0FFF1FE45E8D
:1009C000FE4F808191810E94131BCF91089588234F
:1009D00039F19CEF980F913A18F40E94FF1B0DC05B
:1009E00090E2980F983060F4877091E001C0990F01
:1009F0008A95EAF7892F0E940B0C0E94A90C089592
:100A00009BE5980F933028F480E090E00E94EE1A66
:100A10000895885A8B3120F480E090E00E94131BE7
:100A200008951F93CF93DF93182FEB010E94A70423
:100A3000209741F08FE99FE00197F1F700C0000097
:100A40002197F6CF812F0E94E704DF91CF911F916C
:100A50000895893319F060E070E002C060E570E04D
:100A60000E9411050895882321F00E94050C0E9420
:100A7000A90C0895882321F00E940B0C0E94A90C58
:100A80000895A0E0B0E0E7E4F5E00C945C267C017A
:100A9000162FC72FFC01D581068102950F700E9489
:100AA000FB0B8823F9F0DD23E9F08C2F807F803465
:100AB00061F080E2810F8830A8F08C2F807E803238
:100AC00021F4123078F0002369F08091DE0282FF79
:100AD00009C082E00E94EA0C0E94FB0B91E0D82E34
:100AE000D92601C0D12CCC2EC2948FE0C8228C2DE7
:100AF00090E08C30910508F089C1FC01EA5AFF4F63
:100B00000C9445268C2F807FCF70882311F0C295DE
:100B1000C07FDD2399F0CC2309F464C180E2810F0A
:100B2000883010F0111104C08C2F0E94050C03C0F6
:100B30008C2F0E94150C0E94A90C54C1812F0E9479
:100B4000E704CC2309F462C180E2810F883038F1D8
:100B5000112329F18C2F0E941B0C24C08C2F807F25
:100B6000CF70803211F0C295C07F112319F011307F
:100B700099F13CC08091DE0282FD17C0DD2349F06F
:100B8000CC2329F08C2F0E94050C0E94A90C80E038
:100B90002AC180E00E94E704CC2309F437C18C2FDE
:100BA0000E940B0C0E94A90C31C1DD2349F00023E7
:100BB00009F1013009F02AC18C2F0E942C0C26C1AA
:100BC000011124C18C2F0E943A058C2F0E94380CF1
:100BD0008C2F0E94BD0C1AC1DD2321F0063008F0D5
:100BE00015C108C0053008F011C115C0DD2331F072
:100BF0000111F8C08C2F0E94330508C1002359F061
:100C0000193309F000C1FFEF27EE83E0F1502040D7
:100C10008040E1F7F6C08C2F0E943A05F7C08C2F78
:100C200086958695837019F0813061F0EFC0DD23E1
:100C300021F0812F9C2F937002C080E090E00E94F1
:100C4000EE1AECC0DD2321F0812F9C2F937002C09F
:100C500080E090E00E94131BE1C08C2F837079F537
:100C6000D111D8C0412F429546954770440F440F8B
:100C7000212F2F70042E01C0220F0A94EAF714FFCF
:100C800008C08FE090E001C0880F4A95EAF7809590
:100C900001C080E0C695C695C370822BC23049F072
:100CA00058F4C13019F00E94CA07B4C00E94C407AA
:100CB000B1C00E94D007AEC00E94C107ABC0DD2307
:100CC00019F08C2F817001C08695882309F4A2C089
:100CD000412F429546954770440F440F212F2F70A6
:100CE000042E01C0220F0A94EAF714FF08C08FE017
:100CF00090E001C0880F4A95EAF7809501C080E036
:100D0000C695C695C370822BC23049F058F4C130E5
:100D100019F00E9413087EC00E940D087BC00E943B
:100D2000190878C00E94D60775C0CF70DD2339F04E
:100D30008C2F0E94E807812F0E9433056BC0812F02
:100D40000E943A058C2F0E94F40764C0123F21F1E3
:100D500028F4103F41F0113FC1F040C0133F19F19A
:100D6000143F79F03BC0DD2341F0053008F04EC060
:100D70008C2F8F710E94010849C0063008F046C0D0
:100D8000F7CF8091DE0282FD18C0DD2339F08C2F71
:100D90008F710E94E8073AC0DD23C9F38C2F8F7151
:100DA0000E94F40733C0DD2329F08C2F8F710E943D
:100DB000DF072CC00E94DB0729C0DD2331F063E090
:100DC0008C2F8F710E94CC0C21C081E00E94EA0C14
:100DD0000230E0F082E00E94EA0C18C0DD2331F01E
:100DE0000023A9F2812F0E94A70410C00023B1F2B2
:100DF000193349F49FEFE7EEF3E09150E040F04003
:100E0000E1F700C00000812F0E94E70488EF8C0DFD
:100E1000843020F40E94C81A0E944604DD2089F024
:100E20000E94F70B80FD0DC0F70115820E94F10BA7
:100E30000E94E807C7010E943E070E94F10B0E9432
:100E4000F407CDB7DEB7E8E00C9478260F931F9334
:100E5000CF93DF93EC01688179818D810E94D10865
:100E60008C010E941F080E94B407B801CE010E94A5
:100E70004105DF91CF911F910F910895CF93DF939B
:100E8000FC0124812223D1F0EC010E949203811104
:100E90000FC00E94FB0B882389F08D81882371F09D
:100EA0008091DE0282FF0AC082E00E94EA0C06C046
:100EB000CE010E942607CE010E944B03DF91CF9105
:100EC000089580E090E00E94EE1A80E090E00E9499
:100ED000131B0E94220C0E94A90C08950E94191C49
:100EE0000E94610708950E94120C0E946E070895E7
:100EF00092959F70963079F010F4925001C09A50FC
:100F0000923068F4803F69F018F4883E40F409C0DC
:100F1000843F29F406C0883E20F0813F11F080E034
:100F2000089581E00895FC012481222339F0808115
:100F300091810E94C6080E947807089580E0089574
:100F4000A6E0B0E0E6EAF7E00C9462262696E2E03E
:100F50000C947E26A7E0B0E0E0EBF7E00C9462266C
:100F60002796E2E00C947E26089508950E94B50726
:100F700008950E94B60708950E94B9078093EA0178
:100F800008950E94BC0708959091EA01892B0E9460
:100F9000BC0708959091EA0189230E94BC07089537
:100FA0009091EA0189270E94BC0708950E94CC0213
:100FB0008093E901089580E00E94D607089591E0AA
:100FC00001C0990F8A95EAF7892F0E94D6070895E4
:100FD00021E030E001C0220F8A95EAF78091E90113
:100FE000822B0E94D607089521E030E001C0220F35
:100FF0008A95EAF720958091E90182230E94D6071D
:10100000089521E030E001C0220F8A95EAF780912F
:10101000E90182270E94D60708959091E901892B62
:101020000E94D60708959091E90189230E94D6076E
:1010300008959091E90189270E94D607089508959F
:10104000962F9770A1E001C0AA0F9A95EAF793E056
:10105000769567959A95E1F7FB01EE0FFF1F6E0FEE
:101060007F1FFA01E60FF71F40E050E0682F70E0A5
:1010700090819B01042E02C0369527950A94E2F7D1
:101080002170219529272A23292721934F5F5F4F1C
:101090004330510569F708959B01782F777043E03D
:1010A000969587954A95E1F7FC01EE0FFF1F8E0F8D
:1010B0009F1FF901E80FF91F40E050E080E0219107
:1010C00030E0072E02C0369527950A94E2F721708A
:1010D0003327042E01C0220F0A94EAF7822B4F5FB8
:1010E0005F4F4330510559F70895282F9A3070F417
:1010F0008A3060F4862F622F70E02AE0929F600DA4
:10110000711D112442EC51E00E94200808959A308C
:1011100070F48A3060F4292F90E062EC71E03AE0DC
:10112000239F800D911D11240E944C08089580E09A
:101130000895CF92DF92FF920F931F93CF93DF9387
:101140006C010091E9018091EA01082BC3E0D0E035
:1011500010E0C8010C2E02C0959587950A94E2F71D
:1011600080FD04C02197A8F7F12C07C0FC2EB60122
:101170008C2F0E9405100197A9F38F2DDF91CF913D
:101180001F910F91FF90DF90CF900895CF93DF9341
:10119000EC010E949908BE010E940510DF91CF91D9
:1011A00008951F93CF93DF93EB019091C101992391
:1011B00021F0CB010E94C60813C0882349F0CB015F
:1011C0000E949908182F682FCE010E94750804C04C
:1011D000CB010E948708182FBE01812F0E940510A5
:1011E000DF91CF911F910895E1E0F0E0DF0102C0AF
:1011F000AA0FBB1F6A95E2F7BD01DF0102C0AA0F6B
:10120000BB1F4A95E2F7AD01462B01C0EE0F2A95B0
:10121000EAF7942F9823491302C08E2B0895E09586
:101220008E230895242F462F682F8091E9010E9474
:10123000F4080E94D60708951F93CF93DF93C091BF
:10124000EB0117E08091EC01C817A1F0D0E01C9FE2
:10125000F0011D9FF00D1124E351FE4F20813181DB
:10126000428153816481758186810E94AA072196FB
:10127000C770E8CFDF91CF911F910895209125028B
:101280003091260240912702509128026091290254
:1012900070912A0280912B020E94AA070895CF9391
:1012A000DF9380912B0282958F7009F04EC0809160
:1012B0002A02882309F449C08091EB014091EC0196
:1012C0005091260260912502C0912702D0912802F8
:1012D00077E08417D1F190E0789FF001799FF00DCD
:1012E0001124DF01A351BE4F14962C911497222391
:1012F00049F111962C911197251324C02C91261396
:1013000021C015962C91159721111CC012962D9174
:101310003C9113972C1B3D0B283C310598F4809190
:101320002B028F70806180932B02ED50FE4F8081E5
:101330008F708061808385E292E00E943E070E9468
:101340001C0903C001968770C4CFDF91CF91089527
:101350002091EB019091EC0157E02917A9F030E0C2
:10136000529FF001539FF00D1124E351FE4F718104
:10137000761306C07081781303C07581741306C09C
:101380002F5F3F4F2770E9CF80E0089581E00895F7
:10139000A4E1B0E0EEECF9E00C9458268C0186E074
:1013A000F801DE011F9601900D928A95E1F7F80190
:1013B0008481E58095E2A92E92E0B92E90912902D0
:1013C000911118C0882309F480C1EE20D9F1C80119
:1013D0000E949307F82E8823A9F187E0F801D50130
:1013E00001900D928A95E1F7C5010E949E040E942A
:1013F0004F0998C0F801C080D18082809380F0901E
:101400002A022091270230912802A401421B530B8B
:10141000FF2009F406C1483C510508F0AFC08823FD
:1014200009F455C180912B02282F207F909126022C
:10143000222361F09D1509F462C0C8010E94930740
:10144000811173C0C8010E943E073FC19D1115C0A4
:10145000909125029C1111C0E1100FC08F70806126
:1014600080932B020E943E0985E292E00E943E0793
:1014700080912B02F801868326C1E1103AC040E03A
:101480006D2D8C2D0E94A80940E06D2D8C2D0E94A1
:10149000A809E82E811117C1CF86D88A8F8598892F
:1014A0000E94C608292F22952F70243020F49F70A7
:1014B000223028F009C02A50223080F014C099232D
:1014C00049F0811107C013C0992321F0F8019681DA
:1014D000907F69F0805E883030F409C0803F38F03A
:1014E000815F833020F0C8010E943E07EF2CFE2C64
:1014F000EEC080912B02816080932B02E4C090911A
:1015000025029C119ACFE11098CFF8018683C8017B
:101510000E943E0787E0F801A5E2B2E001900D923B
:101520008A95E1F70E943E09D2C0EE2009F48ACFE5
:1015300020912B02822F82958F7090E002978CF081
:101540008091250290912602998788879B868A86BA
:10155000809129028C871D862E87CE0108960E94D5
:101560003E0787E0F801A5E2B2E001900D928A956E
:10157000E1F70E944F090E943E09A7C090912B02FB
:10158000292F207FA1F4682D9A8A898AA6017A8959
:101590009E2D0E94A00785E292E00E943E0787E010
:1015A000F50111928A95E9F70E943E098CC08823C3
:1015B00009F48DC0809126028D1111C08091250201
:1015C0008C110DC0E1100BC0F8019683C8010E9478
:1015D0003E0787E0F50111928A95E9F778C0C801C6
:1015E0000E949307882309F42DCFEE2009F42ACF17
:1015F00020912B02822F82958F7090E002970CF43D
:10160000B0CF80912502909126029A8389839C8293
:101610008B82809129028D831E822F83CE010196B9
:101620009ECF483C510508F040C0882309F44DC0C6
:10163000FE2CEE2009F406CF809126028D1127C0E2
:10164000809125028C1123C090912B0290FD16C031
:10165000892F82958F70282F30E02115310571F088
:10166000F80196832F30310509F451CF8F5F982F01
:101670009295907F86818F70892B48CF87E0F80103
:10168000A5E2B2E001900D928A95E1F720C0C80171
:101690000E949307811165CF80912B028160809316
:1016A0002B02C8010E943E0712C0682D9A8A898ABF
:1016B000A6017A899E2D0E94A00787E0F50111926C
:1016C0008A95E9F72FCFF12C02C0FF24F3948F2DD8
:1016D0006496ECE00C947426AEE0B0E0E2E7FBE048
:1016E0000C946126288739874A875B876C877D87BA
:1016F0008E87CE0108960E94C809882361F06C8508
:101700006623A9F1288539854A855B857D858E8587
:101710000E94AA072CC087E0FE013896DE011196D0
:1017200001900D928A95E1F76C85662301F1209175
:10173000EC0130E0C9010196877099274091EB01D7
:1017400050E084179507E1F16D8397E0929FD001F7
:10175000939FB00D1124A351BE4FFE01319601900D
:101760000D929A95E1F78093EC010E941C0917E015
:101770008091EB019091EC01891779F1189FC001DC
:10178000112483519E4F0E94C809882331F1E091B2
:10179000EB011E9FF0011124E351FE4F20813181A6
:1017A000428153816481758186810E94AA0780915C
:1017B000EB0190E00196877099278093EB01D8CFD9
:1017C0000E9473071092EC011092EB01E5E2F2E047
:1017D00087E0DF011D928A95E9F72E96E3E00C94ED
:1017E0007D268091540286958695869508958091F0
:1017F00054028770089590915402977081E009F423
:1018000080E0089580918002089590918002892B54
:10181000809380020895809590918002892380931F
:101820008002089510928002089590917F02892B82
:1018300080937F020895809590917F028923809301
:101840007F02089510927F02089508950E94250C4A
:1018500008950E94260C089590915602292F28235E
:10186000821729F0982B909356020E94290C089514
:1018700090915602292F282331F080958923809357
:1018800056020E94290C089580915602882329F05F
:101890001092560280E00E94290C0895CF93C091C7
:1018A000800280917F02C82B80915602882331F0FC
:1018B000C82B0E94381B81110E94440C8C2FCF91A1
:1018C0000895CF93DF93C0910201D09103010E944C
:1018D0004E0C8883C0910201D091030148E050E092
:1018E0006CE472E0CE010E948926892B59F088E0D1
:1018F000FE01ACE4B2E001900D928A95E1F7CE01D1
:101900000E94D51ADF91CF910895CF93DF93C091B4
:101910000001D09101010E944E0C8983C091000109
:10192000D091010140E250E06CE272E0CE010E94F1
:101930008926892B59F080E2FE01ACE2B2E00190E9
:101940000D928A95E1F7CE010E94E01ADF91CF91C6
:1019500008950E947C1C813039F48091DD0287FF5C
:1019600003C00E94850C08950E94610C08950E9496
:10197000250C08950E94B70C089590915502292FC7
:10198000282331F080958923809355020E94BA0C58
:1019900008950E94250C08959091DE0292FF11C0D7
:1019A00098E0899F90011124262B209354020E94D5
:1019B000E807809154028695869586950E94C90C09
:1019C00008950E94E80708951092540280E00E9452
:1019D000C90C0895909154028095892380935402F4
:1019E000282F277069F4981759F09091DE0292FF22
:1019F00007C08695869586950E94F4070E94E40CA0
:101A000008959091DE0292FB222720F9281769F0B1
:101A100080FB92F99093DE028091DD029091DE02CC
:101A20000E94500D82E00E94EA0C08958091DE022F
:101A300082FB882780F991E089270E94010D089593
:101A400081E00E94010D089580E00E94010D08953B
:101A50006FEF7FEF80E090E00E94DB26089580E04A
:101A600090E00E94A726853E9E4F19F40E946E19B1
:101A7000089580E0089582E090E00E949F260895F6
:101A800083E090E00E949F260895682F83E090E015
:101A90000E94BD26089584E090E00E94A726089544
:101AA000BC0184E090E00E94DB260895AB01BC01FC
:101AB0008FE090E00E94CF260895AB01BC0183E146
:101AC00090E00E94CF26089560E070E0CB010E9474
:101AD0005D0D089560E070E0CB010E94560D0E94FC
:101AE000640D0895A8E0B0E0E8E7FDE00C946226FC
:101AF00065EE7EEF80E090E00E94DB2660E082E011
:101B000090E00E94BD2681E08093EA010E94450D8D
:101B100060E074E184E090E00E94DB2660E086E013
:101B200090E00E94BD2660E087E090E00E94BD2624
:101B300040E050E0BA0188E090E00E94CF2660E0EB
:101B400083E290E00E94BD2660E08CE090E00E947D
:101B5000BD2660E08DE090E00E94BD2619821A82C9
:101B60001B821C821D821E821F82188648E050E064
:101B700067E170E0CE0101960E94AD2640E050E0A2
:101B8000BA018FE190E00E94CF2680E00E94871981
:101B90000E94BC190E946A0D2896E2E00C947E26F1
:101BA0000E94720D0895682F8EE090E00E94BD267D
:101BB0000895A6E0B0E0EFEDFDE00C9460260E94F1
:101BC0002D1D8C01809181029091820208171907C6
:101BD00081F019821A820E942D1D682F49815A8135
:101BE000792F80E090E00E946B04109382020093B2
:101BF00081022696E4E00C947C260E94391D6093B5
:101C00009B0270939C0280939D0290939E0260932E
:101C10009702709398028093990290939A02089584
:101C200081E0089581E008950E94120E08950895BC
:101C30000E94170E08950E94170E08950E941B0E11
:101C400008950E94170E08950E94170E089585EFBB
:101C500090E10E9470120E94240E0E94C802089512
:101C60000E94180E0E94170E08950E942F0D8111D8
:101C700002C00E94D00D0E943B0D80939F020E94E3
:101C80004B0D9093DE028093DD020E94B0140E94FF
:101C9000400D0E94C1078091E9010E94CC02089585
:101CA0000E94241D0E94CC190E94C8110E94350E6A
:101CB0000E943F0480E00E94BD120E941E0E089503
:101CC000A6E0B0E0E6E6FEE00C9456260E94100E78
:101CD000811104C00E94D90D10E063C00E94DE1182
:101CE00023E8E22E22E0F22E5701D12CF5010191DA
:101CF00011915F018D2D0E940A1180279127D394A5
:101D0000FAE0DF1619F0892B89F302C0892B11F351
:101D100080919F0281FD0E9413110E94140E782E63
:101D200010E066246394812F0E940A114C01F70190
:101D3000A080B180A826B926A114B10449F100E021
:101D4000CC24C394D12CC5018C219D21892BC1F0B9
:101D50007720B1F009831A830E942D1D9C838B8309
:101D60006D8221E0C4018C219D21892B09F420E0A2
:101D700049815A816B817C818D81922F0E946B04F5
:101D80000F5FCC0CDD1C0A30F1F6F70191828082E6
:101D90001F5FF2E0EF0EF11C1A3029F60E94FD0DD4
:101DA00011E00E94651411110E9422130E94520436
:101DB0002696EEE00C9472261F93CF93DF930E9439
:101DC0000A10EC01C11580E5D807E8F5C11590E4CB
:101DD000D90708F0A8C0C03ED10530F5CD3CD105EB
:101DE00008F094C0C83AD10578F4C53AD10508F096
:101DF00083C0C130D10509F47CC008F4F2C0C430FE
:101E0000D10508F0F1C0EDC0C33CD10508F0E9C030
:101E1000C85AD0E0CC0FDD1FCB5ADE4F0990D881D5
:101E2000C02DCE019464E1C0C11580E2D80708F04E
:101E3000CBC0C11591E0D90708F06BC0C83ED105F1
:101E400008F4D2C0CEC0C03682E5D80728F5C03429
:101E500092E5D90708F079C0C03282E5D80708F0CA
:101E60006CC0C11592E5D90708F481C04C2F469586
:101E7000469580E2489FA0011124C37021E030E024
:101E8000C90102C0880F991FCA95E2F7EA01C82B61
:101E9000D92BCE019D68A9C0C03A82E5D807B8F415
:101EA0008C2F8F71C03892E5D90708F07BC08695DA
:101EB000869590E2899F90011124C37081E090E0A3
:101EC00002C0880F991FCA95E2F79A6868C0C03CA3
:101ED00082E5D80708F46DC0C03E92E5D90708F046
:101EE00080C0CF71DD27DC2FCC27CE01806F906AB8
:101EF0007CC081E090E079C0C55AD0E0C557DE4F84
:101F00008881C82FD0E0CE0190646FC0CE0190656B
:101F10006CC08D2F0E94A610182FCE0199270E9409
:101F20000A101F715CC0CE0199270E940A10CC27AD
:101F3000DF70D06A8C2B9D2B58C0CF71D0E0DC2F86
:101F4000CC27CE01816F906A50C08C2F8F718695FF
:101F5000869590E2899F90011124C37081E090E002
:101F600002C0880F991FCA95E2F79C6818C08C2F91
:101F70008F710E94A61095E0D695C7959A95E1F7C6
:101F8000CF70D0E0DC2FCC27282F30E084FF05C0B5
:101F900084E0220F331F8A95E1F7D069CE01822BAE
:101FA000932B23C090E0D82FCC27CE01846F906A6A
:101FB0001CC08C2F8F710E94A6108F7190E0D82FBB
:101FC000CC27CE01906211C08D2F8F710E94A61078
:101FD000182FCE0199270E940A101F719062912B31
:101FE00004C080E090E001C0CE01DF91CF911F914D
:101FF00008957A3038F46A3028F4462F672F0E940B
:102000006215089580E090E008950E94F90F0E9403
:10201000DC0E08958238910569F1B0F481339105A1
:1020200009F475C048F48932910509F467C08A3211
:10203000910509F471C008958533910509F459C0DB
:1020400089339105B9F00895833E910589F138F4FB
:10205000803E9105D1F0823E910529F10895863E9A
:102060009105C9F1873E9105D9F1843E910509F0AA
:102070006CC027C02091DD0220FD57C021FD55C056
:102080002091DE0223FD5BC008958091DD0280FD7A
:1020900048C08091DE0280FF48C08091DD0284FD4F
:1020A00046C083EE51C08091DD0282FF3CC0F5CF77
:1020B0008091DD0282FD37C08091DE0280FD35C057
:1020C000ECCF8091DE0281FF36C08091DD0284FD7D
:1020D0002EC087EE39C08091DD0283FF2AC0F5CF84
:1020E0008091DD0283FD25C08091DE0281FD23C049
:1020F000ECCF8091DD0285FD22C01FC08091DD0202
:1021000085FD1BC08091DE0283FF19C00AC080914B
:10211000DD0286FD16C017C08091DD0286FD13C06A
:1021200010C089E311C082EE0FC080EE0DC080E0C8
:102130000BC086EE09C084EE07C085E305C089E2C6
:1021400003C08AE201C081E390E008959091DD022E
:1021500092FF10C041E0282F2471243009F040E0A4
:1021600031E0282F2871283009F030E0431711F0B2
:102170002CE0822793FF10C041E0282F24712431E6
:1021800009F040E031E0282F2871283109F030E0D3
:10219000431711F02CE082273091DE0230FF10C08F
:1021A00051E0282F2171213009F050E041E0282F23
:1021B0002871283009F040E0541711F029E08227F7
:1021C00031FF10C041E0282F2171213109F040E09A
:1021D00031E0282F2871283109F030E0431711F041
:1021E00029E0822794FD877E089580E00895CF93AB
:1021F0009C01205E32452032310540F4FB01C5814F
:10220000C11105C08F710E94600301C0C1E08C2F15
:10221000CF910895E82FF0E0EE0FFF1FED50FD4F36
:10222000808191810895089580EA8A95F1F7089553
:1022300000C008950E941411089508950E941D1170
:1022400008950E941E1108950E941D1108950E9474
:1022500024110895F894E82FE295EF70F0E031A191
:10226000282F2F7081E090E001C0880F2A95EAF7AF
:10227000982F9095932391A392A1892B82A3789470
:1022800008950F931F93CF93DF93C8E9D1E089910D
:102290008F3F11F00E942A1181E0C23AD807B9F7A6
:1022A000CEE8D1E008E911E089918F3F11F00E945A
:1022B0002A110C171D07C1F7DF91CF911F910F91C4
:1022C0000895A0E0B0E0E7E6F1E10C945B268C0114
:1022D000C62FD0E0CE0188569E4F6C01FC01908144
:1022E0009F3F09F450C0B62EF894E92FE295EF70A5
:1022F000F0E081A19F7021E030E001C0220F9A95AB
:10230000EAF7822B81A382A12095282322A3789427
:102310000E941811EEE8F1E048E951E021E030E0D8
:10232000E12CF12C61916F3F89F0A62FA295AF703F
:10233000B0E090968C9190E06F7002C09595879573
:102340006A95E2F780FD02C0C90102C080E090E01A
:10235000E82AF92A220F331F4E175F0719F7F601F3
:1023600080818F3F11F00E942A1161E0E114F10495
:1023700009F460E08B2D0E941A11CC0FDD1FC00FF5
:10238000D11FF982E882CDB7DEB7E9E00C94772659
:102390000E94411184E1E3EFF2E0DF01982F1D92EA
:1023A0009A95E9F7EFEDF2E0DF011D928A95E9F7E2
:1023B0008AE00E9419120E9427110895A4E1B0E05A
:1023C000E4EEF1E10C945F268E010F5F1F4F84E174
:1023D000F80111928A95E9F7F12C6F2DC8010E943E
:1023E0006111F394FAE0FF12F8CF44E150E0B80134
:1023F0008FED92E00E94892621E0009709F420E009
:10240000892B41F084E1F801AFEDB2E001900D922B
:102410008A95E1F74AE063EF72E08FED92E00E9467
:102420001A12182F0E942111812F6496E5E00C9456
:102430007B260895EF92FF920F931F93CF93DF9324
:102440007C018B01C42F222351F081E08093A202F2
:102450000E942D1D9093A1028093A00204C0809140
:10246000A202811102C080E01CC08091A002909164
:10247000A1020E94451D0597B0F3D0E0CC0FDD1FEF
:10248000AE01B701C8010E948926892B39F0AE013F
:10249000B701C8010E94962681E001C080E0109239
:1024A000A202CDB7DEB7E6E00C947A260E94600E59
:1024B00008950E94C41C0E94A3200E94270E0E941F
:1024C000BD200E94500E0E94CA200E94CF200E9470
:1024D00056120E94E9200E94681F0E94300EF5CF1C
:1024E0009093BB018093BA010895AB0124E630E0DC
:1024F000BC0188E70E94311E21E0892B09F020E011
:10250000822F0895AB0124E630E0BC0188E70E94E9
:102510007C1E21E0892B09F020E0822F08950F9383
:102520001F939B0104E610E0AC0160E488E70E9481
:10253000C81E21E0892B09F020E0822F1F910F9106
:1025400008950E94FC1D089508950E94A412089504
:10255000E7E0F3E080E092E0DF019C011D92215072
:102560003040E1F7F0930C05E0930B058FEF9FEF00
:102570009093C9028093C8020895CF930E94A51238
:102580000E94A4128093C40280FD02C080E801C0B2
:1025900080E28093C3020E94A1126BE070E08BEF97
:1025A00092E00E948212811102C0C0E031C080918D
:1025B000C40265E070E081FD03C086EF92E002C0D6
:1025C00081EF92E00E948212882379F36DE070E03F
:1025D00084EE92E00E948212C82F882331F30E9479
:1025E000391DDC01CB01805A9541AF4FBF4F80931D
:1025F000070590930805A0930905B0930A050E946A
:10260000A81281E08093C7028093C6021092C5028F
:102610008C2FCF9108952091C30236E0839FC00193
:102620001124629F800D911D1124811522E09207D3
:1026300014F080E090E0895F9C4F90930C058093AC
:102640000B0508958091C7028823F9F00E94391D77
:10265000DC01CB01805A9541AF4FBF4F80930705F6
:1026600090930805A0930905B0930A058091C602CE
:1026700081110BC062E070E082EE92E00E94821253
:10268000882319F081E08093C6028091C6020895E4
:10269000A4E0B0E0EEE4F3E10C9452262091C802ED
:1026A0003091C902232B09F4EDC09091C702992300
:1026B00009F4E8C09091C5029111E4C0082F0E946E
:1026C0002213F12C10E0AA24A394B12CB3E0EB2E3A
:1026D00080E2D82E8091C8029091C902009709F437
:1026E000D1C0F110CDC0212E312C9501012E02C098
:1026F000220F331F0A94E2F73A83298328233923D0
:10270000232B11F41F5FEFCF2091C402C101F5E02C
:10271000880F991FFA95E1F720FD13C0880F892FC4
:10272000881F990B9195912F9295990F9076909380
:10273000060180930901915E9093070180930A013D
:1027400011C075E0969587957A95E1F7880F880F07
:10275000880F8093060110920901895F8093070119
:10276000E0920A0167E070E084E091E00E94751257
:10277000882309F487C08091C40280FD1FC0C10175
:1027800065E0880F991F6A95E1F760E270E0895F64
:102790009C4F0E948F12882309F474C069817A814A
:1027A000609570958091C8029091C9026823792341
:1027B0007093C9026093C802F3948CCFA3EAB2E08D
:1027C000ED2D1D92EA95E9F755E0220C331C5A9540
:1027D000E1F726EA31E03C832B8382EA91E0AB818A
:1027E000BC812D91BC83AB83FC013191CF01A10150
:1027F000430F511DBA01695F7C4F2B0130E02D550D
:102800003D4FF90147E0942EAF01421B530B7A2C48
:1028100001C0770C4A95EAF7B201812CDB01CD901B
:10282000BD01C720492D48194770642E042E000CA5
:10283000550BBC2D01C0BB0F6A94EAF76B2E519566
:10284000419551094770552701C0C6944A95EAF74A
:102850006C28C0806C286082839448E08412DECFAC
:102860009A9431966FEF9612CFCFAB81BC81AA5A62
:10287000B14009F0B4CF60E270E083EA92E089CF22
:10288000011131CF2496E2E10C946E268091C702AB
:102890009091C602882389F0992369F062E070E084
:1028A00080EE92E00E948212811103C08091C602E4
:1028B00008951092C6029091C60281E0892708957A
:1028C00081E008950E94601408950F931F938091F2
:1028D000C702882321F160E080E00E940B130E9470
:1028E000621480E00E9448138091C6028823B9F0E8
:1028F0000E94391D009107051091080520910905D6
:1029000030910A05DC01CB01801B910BA20BB30BAC
:102910008F3F9F4FAF4FBF4710F40E9446141F9147
:102920000F9108950E94280D089580E00E940A11D9
:10293000817008950E94DE112FEF86E791E021500B
:1029400080409040E1F700C000000E94DE110E942C
:102950009514882321F00E9492140E947A1D0895F4
:102960000E949A14089584E0089550E0440F551F82
:1029700024E1629F400D511D11249A0168EC869F4D
:10298000200D311D1124C901889608950F931F93BE
:10299000CF93DF938430A0F46A3090F44A3080F40F
:1029A0000E94B5148C010E949F2690E0D82FCC275E
:1029B000C80101960E949F269E01282BC90102C0D2
:1029C00080E090E0DF91CF911F910F9108950F93D8
:1029D0001F93CF93DF93843080F46A3070F44A30D1
:1029E00060F4E9010E94B5148C016D2F0E94BD2690
:1029F0006C2FC80101960E94BD26DF91CF911F91D7
:102A00000F9108951F93CF93DF93D0E0C0E010E0C3
:102A1000412F6C2F8D2F0E94DA029C01412F6C2FC9
:102A20008D2F0E94E7141F5F1A3091F7CF5FCA30D5
:102A300071F7DF5FD43051F7DF91CF911F91089587
:102A4000EF92FF920F931F93CF93DF93EA017A01E6
:102A5000E60EF71E8C01C8018896CE15DF0569F0D9
:102A6000003223E0120720F40E949F26888301C0D1
:102A7000188221960F5F1F4FEECFCDB7DEB7E6E08D
:102A80000C947A26EF92FF920F931F93CF93DF93CC
:102A9000EA017A01E60EF71E8C01C8018896CE1570
:102AA000DF0559F0003223E0120718F468810E9414
:102AB000BD2621960F5F1F4FF0CFCDB7DEB7E6E002
:102AC0000C947A26843038F46A3028F44A3018F4AA
:102AD0000E94C614089580E090E0089580E1089572
:102AE00088EB90E00895EF92FF920F931F93CF939E
:102AF000DF93EA017A01E60EF71E8C01C801885BBC
:102B00009C4FCE15DF0561F0083B110520F40E94B3
:102B10009F26888301C0188221960F5F1F4FEECF3A
:102B2000CDB7DEB7E6E00C947A26EF92FF920F93D2
:102B30001F93CF93DF93EA017A01E60EF71E8C0113
:102B4000C801885B9C4FCE15DF0551F0083B11058D
:102B500018F468810E94BD2621960F5F1F4FF0CFA9
:102B6000CDB7DEB7E6E00C947A26CF93DF93C8E4C6
:102B7000D3E060E0CE010E94BD262196C11584E01D
:102B8000D807B9F7DF91CF910895A8E0B0E0EBEC5A
:102B9000F5E10C945826F82E8FE08F1508F474C0D8
:102BA0008FEF93E00E949F2681116EC008E413E02E
:102BB000FF2071F0011594E0190709F465C0C80100
:102BC0000E949F26811101C0FA940F5F1F4FF0CF22
:102BD000FE0131966F0188E011928A95E9F778013C
:102BE000FFEFEF1AFF0AC8010E949F2689831A820D
:102BF000882309F449C0813009F040C0580182E0BF
:102C0000A80EB11CC7010E949F268A838823E1F188
:102C10009FEF980F933060F4780193E0E90EF11C78
:102C2000C5010E949F268B83882371F11C8226C0D8
:102C3000843019F54E01E3E08E0E911C02E010E0A5
:102C40007501FFEFEF1AFF0AC5010E949F26F401EC
:102C500081934F018823C1F08C3741F4E2E0F0E02A
:102C6000EC0FFD1FE00FF11F108208C00F5F1F4F18
:102C700057010730110521F707C0750160E0C60153
:102C80000E940E188701ABCF2896ECE00C947426B6
:102C9000CF93DF9386319C4709F5EB010E94020C2C
:102CA0009D81992371F08A7A91E009F490E09093E4
:102CB000CA02811102C089E201C085E30E94E51BBE
:102CC00009C08091CA02811102C089E201C085E376
:102CD0000E94FF1B0E94A90C80E001C081E0DF91EF
:102CE000CF910895CF93DF93FC01DB0115968C9172
:102CF000882309F4DDC09F0130572332310508F0E5
:102D0000D8C0EF010E944B0D9093DE028093DD024C
:102D1000FE01E150F047E232F10520F4EE59FF4F99
:102D20000C9445268091DD028160AAC08091DE026C
:102D30008860B2C08091DD028260A2C08091DD0215
:102D400020C08091DD0288609BC08091DE021EC0A1
:102D50008091DE028260A0C08091DD02806190C01F
:102D60008091DD0280628CC08091DD02806488C029
:102D70000E9473078091DD02806882C08091DD022D
:102D8000886084607DC08091DE028260816084C042
:102D90008091DD028E7F74C08091DE02877F7CC0CF
:102DA0008091DD028D7F6CC08091DD0220C080911A
:102DB000DD02877F65C08091DE021EC08091DE0249
:102DC0008D7F6AC08091DD028F7E5AC08091DD02C6
:102DD0008F7D56C08091DD028F7B52C00E947307A9
:102DE0008091DD028F774CC08091DD02877F8B7FE1
:102DF00047C08091DE028D7F8E7F4EC08091DD02C4
:102E000082FB222720F991E0922790FB82F990FB28
:102E100083F936C08091DE02982F909591708E7F55
:102E2000892B90FB81F938C08091DD0286FB222737
:102E300020F991E0922790FB86F922C00E94730747
:102E40008091DD0287FB222720F991E0922790FBF9
:102E500087F916C081E001C080E00E94D30D1EC03A
:102E60008091DD0284FB222720F991E0922790FBDC
:102E700084F906C08091DD02982F909590FB80F92F
:102E80008093DD020BC08091DE0283FB222720F9B4
:102E900091E0922790FB83F98093DE028091DD021E
:102EA0009091DE020E94500D0E94730780E001C0E5
:102EB00081E0DF91CF9108958F929F92BF92CF9240
:102EC000DF92EF92FF920F931F93CF93DF93E82F40
:102ED000F0E0EA5FFC4FB490282F269526952695C2
:102EE00030E0F901EA55FC4FE4908770F12C082E90
:102EF00002C0F594E7940A94E2F791E0E922FF24F6
:102F0000F901EA56FC4FC490D12C082E02C0D5948A
:102F1000C7940A94E2F7E1E0CE22DD24F901EA57F2
:102F2000FC4FC491D0E002C0D595C7958A95E2F7D1
:102F3000C170DD27062F10E0E114F10471F081EE7D
:102F40000E94A704C801009741F0EFE9FFE0319724
:102F5000F1F700C000000197F6CFC114D10439F495
:102F60004801B8018B2D0E941105C8010EC086EEE4
:102F70000E94A704C801009799F3EFE9FFE0319799
:102F8000F1F700C000000197F6CF009741F0EFE99C
:102F9000FFE03197F1F700C000000197F6CFCD2890
:102FA00019F5EF2879F081EE0E94E704011511056B
:102FB00049F08FE99FE00197F1F700C00000015050
:102FC0001109F4CFCD2BF1F08CE20E942905811478
:102FD0009104C1F0EFE9FFE03197F1F700C0000084
:102FE000F1E08F1A9108F3CF86EE0E94E704C80142
:102FF0000097B9F2EFE9FFE03197F1F700C0000068
:103000000197F6CFDF91CF911F910F91FF90EF9035
:10301000DF90CF90BF909F908F900895EF92FF9296
:103020000F931F93CF93DF93EC01162F0AE0888153
:10303000882309F457C0813009F04FC0898181305D
:1030400041F47E0182E0E80EF11C8A810E9429058C
:1030500009C0823049F47E01E2E0EE0EF11C8A8163
:103060000E94A704E7012DC0833041F47E01F2E005
:10307000EF0EF11C8A810E94E704F4CF843011F036
:1030800021961FC02A81229680E090E030E02053F4
:1030900031092A30310558F4089FA001099F500DCD
:1030A0001124C901840F951F21962881EFCF009725
:1030B00041F0EFE9FFE03197F1F700C00000019720
:1030C000F6CF812F90E0009759F0EFE9FFE03197BC
:1030D000F1F700C000000197F6CF612F0E945C1746
:1030E0002196A5CFCDB7DEB7E6E00C947A260F93F4
:1030F0001F93CF93DF93C42FD22FFC0185818823A8
:10310000B1F04093CD020E942D1D9093CC0280938C
:10311000CB0280E28C0F883008F04DC0C77081E090
:1031200001C0880FCA95EAF70E94330544C0809118
:10313000CD02481330C08091CB029091CC020E9406
:10314000451D883C910538F510E21D0FCD17B9F0EB
:1031500080E28C0F883040F4C77081E001C0880F96
:10316000CA95EAF70E943A05183010F581E09D2FC4
:10317000977001C0880F9A95EAF70E943305802F57
:103180000E9429051830B8F4D77081E001C0880F7B
:10319000DA95EAF70AC080E28C0F883060F4C770D5
:1031A00081E001C0880FCA95EAF70E943A0503C082
:1031B000802F0E942905DF91CF911F910F910895D3
:1031C0000F93FC01E851FC47E730F10590F5CB0186
:1031D000EC57FF4F0C94452606E221EE41EE6AE1E2
:1031E0007CE723C007E225EE45EE6BE17CE71DC0DE
:1031F00006E221EE40EE68E17CE717C007E225EE2B
:1032000044EE69E17CE711C006E221EE42EE6CE19A
:103210007CE70BC007E225EE46EE6DE17CE705C0DA
:1032200008E221E045EE6EE17CE70E94771880E03D
:1032300008C0FB018581882319F01092CD0201C0DE
:1032400081E00F9108951F93CF93DF9387372CE789
:10325000920721F088379C4759F031C0FB01C581A6
:10326000CC2319F00E94651909C00E94651918C085
:10327000FB01C581CC2391F00E9468190E94E807E8
:103280000E946B19D82F0E946819C82F0E946519D7
:103290004D2F6C2F0E941209C0E012C00E946819C5
:1032A0000E94F4070E946B19182F0E946819D82FEA
:1032B0000E946519412F6D2F0E94120901C0C1E0C3
:1032C0008C2FDF91CF911F91089580910D0108956A
:1032D00080910C01089580910B01089584E290E0A3
:1032E0000E949F26853281F485E290E00E949F260D
:1032F000813051F486E290E00E949F2691E0843173
:1033000009F090E0892F01C080E081700895CF938B
:10331000C82F811102C06FEF01C065E284E290E026
:103320000E94BD26C11102C06FEF01C061E085E2BD
:1033300090E00E94BD26C11102C06FEF01C064E1A0
:1033400086E290E00E94BD26CF910895089587E21D
:1033500090E00E949F26682F70E080E090E0089542
:103360000895CF93C62F0E94B0196C2F87E290E08A
:103370000E94BD26CF91089580E00E94871960E0E9
:1033800070E0CB010E94B1190E9402150E94B51590
:1033900081E00E94871908950E94A6190E94A7192A
:1033A0000E94B0190E946E19811102C00E94BC19BE
:1033B000089508959C01FB018581882351F0A9019E
:1033C00057574038510530F4C9010E94C51580E0B7
:1033D000089581E008952FEFFC01208308950E9455
:1033E000EB19089580E00895A0E0B0E0EAEFF9E17C
:1033F0000C945A26EC01D62E0E94F2198111BEC0FF
:10340000E8818E2F90E0FC013197E331F10508F05F
:10341000AFC0E557FF4F0C94452619828CE06BC076
:103420008981823089F030F4813009F0A1C00E9496
:10343000391D0CC0833079F0843009F099C01A82AC
:103440001B821C821D8296C00E94A7199A838B83BF
:103450007C836D838FC0CA807E0100E010E0AC2CBD
:10346000B12CC501800F911F0A9708F083C08C2DE5
:10347000800F0E940A11F701938384830F5F1F4F0F
:10348000F2E0EF0EF11C0E30110559F773C089817F
:10349000823039F0853009F06BC08A810E94D919D9
:1034A00069C06A817B818C819D810E944B260E942C
:1034B000B11960C04B816A8189810E94C6149C83C6
:1034C0008D8358C02C813D813227232732274B81A1
:1034D0006A8189810E94E7144DC00E9402154AC08A
:1034E0006D2DCE010E94EF1945C00E946E1524C0BB
:1034F0000E94701599838A833DC06B8170E0898139
:103500009A81AE014C5F5F4F9827892798270E94C8
:10351000731530C06B8170E089819A81AE014C5F78
:103520005F4F9827892798270E94951523C00E94EE
:10353000B51520C00E94B31489831CC06B8170E054
:1035400089819A81AE014C5F5F4F98278927982720
:103550000E9420150FC06B8170E089819A81AE01B5
:103560004C5F5F4F9827892798270E94421502C019
:103570008FEF88836D2DCE010E945F1FCDB7DEB720
:10358000EAE00C9476269093D3028093D2020895B9
:10359000E091D202F091D302309729F00190F081AE
:1035A000E02D0995089580E00895E091D202F09110
:1035B000D302309721F00280F381E02D0995089520
:1035C000E091D202F091D302309739F026E0DC018D
:1035D0002C930480F581E02D09950895A3E0B0E0D7
:1035E000E4EFFAE10C9462262091D0023091D102EE
:1035F00028173907A1F09093D1028093D002E0916F
:10360000D202F091D302309751F023E029839B83BB
:103610008A830084F185E02DCE01019609952396D9
:10362000E2E00C947E26A3E0B0E0E9E1FBE10C943B
:1036300062262091CE023091CF0228173907A1F0DF
:103640009093CF028093CE02E091D202F091D30208
:10365000309751F024E029839B838A830084F1858D
:10366000E02DCE01019609952396E2E00C947E268A
:10367000CF93DF93C0910201D091030122960E9463
:103680007C1C813059F48091DD0287FF07C0C09116
:103690000001D091010122969EE101C096E080E0F8
:1036A000915028F029912223D9F38F5FF9CFDF9130
:1036B000CF910895CF93882329F1C82F0E947C1CB5
:1036C000813011F58091DD0287FF1EC08C2F869519
:1036D000869586958E31B0F4E0910001F09101015C
:1036E000E80FF11D2281822F90E0C77021E030E0C9
:1036F00002C0220F331FCA95E2F72823392381E045
:10370000232B89F480E00FC0809102019091030186
:10371000FC01329608962191C21721F0E817F907AB
:10372000D1F7F0CF81E0CF9108959C01FC01329652
:103730009FEF80E04191461789F09F3F19F44111B6
:1037400001C0982F8F5F8630A9F79F3F39F0F901AC
:10375000E90FF11D97FDFA956283089508959C0184
:103760002A5F3F4FFC014281461301C0128201963D
:1037700082179307B9F70895262F26952695269543
:103780002E3168F4FC01E20FF11D677021E030E09A
:1037900001C0220F6A95EAF78281282B22830895BF
:1037A000262F2695269526952E3170F4FC01E20FE2
:1037B000F11D677021E030E001C0220F6A95EAF741
:1037C00020958281282322830895CF93C82F0E94B9
:1037D0007C1C6C2F813059F48091DD0287FF07C07B
:1037E00080910001909101010E94BC1B06C0809154
:1037F0000201909103010E94951BCF910895CF93F0
:10380000C82F0E947C1C6C2F813059F48091DD02FE
:1038100087FF07C080910001909101010E94D01B99
:1038200006C080910201909103010E94AF1BCF91CD
:1038300008950E947C1C813059F48091DD0287FF3D
:1038400007C0E0910001F091010132968EE106C0BF
:10385000E0910201F0910301329686E0DF011D92B2
:103860008A95E9F7089508950E94331C089583E02E
:103870008093110160910E0170910F0180911001F0
:10388000909111010E94341C0895811102C081E0C1
:1038900001C082E08093110160910E0170910F01CF
:1038A00080911001909111010E94341C08950E9492
:1038B000451C089581E08093110160910E01709183
:1038C0000F0180911001909111010E94341C089504
:1038D0000E945A1C089591E0811101C090E09093DC
:1038E000100160910E0170910F0180911001909173
:1038F00011010E94341C0895809110010895809355
:103900000F0160910E0170910F0180911001909153
:1039100011010E94341C089580910F010895809335
:103920000E0160910E0170910F0180911001909134
:1039300011010E94341C089580910E01089508958C
:103940000E949F1C08950E94A01C08950E949F1C25
:1039500008950E949F1C08950E949F1C0895CF9374
:103960000E94A91C0E94DE110E94A61CC0E08C2FA0
:103970000E940A11892B29F4CF5FCA30C1F780E079
:1039800001C081E0CF91089585B7806885BF85B774
:10399000806885BF08951F920F920FB60F92112471
:1039A0008F939F93AF93BF938091D402811113C0E3
:1039B00080910D0590910E05A0910F05B091100515
:1039C0004196A11DB11D80930D0590930E05A09306
:1039D0000F05B0931005BF91AF919F918F910F90FC
:1039E0000FBE0F901F90189580911505843031F10E
:1039F0000E94FE031092D40220E488E190E00FB60A
:103A0000F894A895809360000FBE2093600083B760
:103A1000817F846083BF83B7816083BF78948895FA
:103A200083B78E7F83BF0FB6F894A895809160000E
:103A3000886180936000109260000FBE08950E941C
:103A400073070E940504089582E084BD93E095BD4C
:103A50009AEF97BD80936E0008952FB7F8948091E8
:103A60000D0590910E05A0910F05B09110052FBF87
:103A700008952FB7F89460910D0570910E0580910F
:103A80000F05909110052FBF08959C014FB7F89432
:103A900080910D0590910E05A0910F05B091100534
:103AA0004FBF821B930B089578941F920F920FB60D
:103AB0000F9211248F939F93AF93BF9380910D0525
:103AC00090910E05A0910F05B09110050196A11DD2
:103AD000B11D80930D0590930E05A0930F05B09333
:103AE0001005BF91AF919F918F910F900FBE0F90D6
:103AF0001F90189581E08093E00080E28093D800C9
:103B00001092C9008FE19EE40197F1F700C0000018
:103B100087E090EBDC0180931E0590931F05A09336
:103B20002005B09321059CE088E10FB6F894A89594
:103B3000809360000FBE90936000FFCF9CE088E10F
:103B40000FB6F894A895809360000FBE9093600024
:103B5000FFCFEF92FF920F931F93CF93DF93182F16
:103B6000EB011092BC0084EA8093BC000E942D1DE2
:103B70007C018091BC0087FD0DC0CF3F8FEFD8073F
:103B8000C1F3C7010E94451DC817D90790F78EEFF2
:103B90009FEF2DC08091B900887F883041F08091DF
:103BA000B900887F803119F08FEF9FEF20C010930C
:103BB000BB0084E88093BC000E942D1D8C01809185
:103BC000BC0087FD0BC0CF3F8FEFD807C1F3C80102
:103BD0000E94451DC817D90790F7D9CF8091B90029
:103BE000887F883111F08034F9F680E090E0CDB71D
:103BF000DEB7E6E00C947A261092B9008CE0809350
:103C0000B80008950F931F93CF93DF93EB01809338
:103C1000BB0084E88093BC000E942D1D8C01809124
:103C2000BC0087FD0DC0CF3F8FEFD807C1F3C8019F
:103C30000E94451DC817D90790F78EEF9FEF0CC063
:103C40002091B900287F81E090E0283211F480E0D3
:103C500090E0919581959109DF91CF911F910F91FE
:103C60000895A0E0B0E0E7E3FEE10C945726782E3B
:103C7000B62EA72E6A0189010E942D1D4C01043128
:103C8000110558F00F3F8FEF180751F0C80164E19C
:103C900070E00E943126EB0105C0C1E0D0E002C017
:103CA000C5E0D0E0BE01872D0E94A91D7C0197FDD3
:103CB00005C0CB2DDA2DCC0EDD1E12C00F3F8FEFCD
:103CC000180781F3C4010E94451D0817190750F712
:103CD000F0CFF7FC08C0B80189910E94021E7C0158
:103CE000CC15DD05B1F784E98093BC00C701CDB7E1
:103CF000DEB7EDE00C947326A0E0B0E0E2E8FEE170
:103D00000C945726782EEB016A0189010E942D1D23
:103D10004C010431110558F00F3F8FEF180759F08F
:103D2000C80164E170E00E9431265B0107C0AA244B
:103D3000A394B12C03C085E0A82EB12CB501872D2A
:103D40000E94A91D7C0197FD03C0CC0EDD1E14C08E
:103D50000F3FEFEF1E0791F3C4010E94451D0817A6
:103D6000190760F7F2CFF7FC0AC0FE018491B80191
:103D70000E94021E7C012196CC15DD05A1F784E985
:103D80008093BC00C701CDB7DEB7EDE00C9473267D
:103D9000A0E0B0E0EEECFEE10C945626682E762E04
:103DA0005A0169010E942D1D4C010431110558F082
:103DB0000F3F8FEF180751F0C80164E170E00E94D7
:103DC0003126EB0105C0C1E0D0E002C0C5E0D0E083
:103DD000BE01862D0E94A91D7C0197FF0BC00F3FDD
:103DE0008FEF1807A9F3C4010E94451D0817190792
:103DF00078F713C0B801872D0E94021E7C01E501EF
:103E0000CA0CDB1CCC15DD0541F0F7FC06C0B8017F
:103E100089910E94021E7C01F5CF84E98093BC0049
:103E2000C701CDB7DEB7EEE00C94722608959B0172
:103E3000909115059430F1F48F708093E9008FEF25
:103E40009091E800815095FD06C095ED9A95F1F7A7
:103E500000008111F5CF8091E80085FF0BC0BA0109
:103E6000C90140E050E00E945E218091E8008E7719
:103E70008093E800089543E050E0BC0184E00E9494
